S123C0000F8E07FFCE1000A60184F78A87A701A60984C3A7098601A7261C24408630A72BBE
S123C0208610A72C862CA72DCC0824FD0834FD0836CC0838FD0848FD084ACC00B4FD08066E
S123C040CC0000FD0802FD080AFD080CFD080FFD0811B70815B7080EB70813B70814B708BA
S123C06016B70817B70818B70819B7081AB7081BB70865B70866B70851B70852CE1000A680
S123C0802E84202704A62F20F60EBDC3A1BDC3B1BDC3FEBDC415BDC42CBDC445BDC37DBD13
S123C0A0C3EABDC4E58A20BDC575860AB7085CBDC4E58420270B7A085C26F4CC00027EC4D9
S123C0C0CB8609C607BDC4988607C647BDC4988606C60EBDC4988605C600BDC498BDC3EF17
S123C0E0BDC415BDC460BDC3A1BDC3B17D081527EFFC0806FD0808CC0000FD0806BDC37DD8
S123C1007D081526FB7D081626037EC1F9BDC3EA7D081926037EC1FC7D081A27037EC1FCF4
S123C1207C081A7D08652765FE080C09FF080C2609FE080AFF080C7A080EFE085D09FF0864
S123C1405D264AFE0861FF085DFE080AFF080C8605B7080EBDC3A1B6080527188101270AF2
S123C160810227068103270C2023B6085181C0271C4C2006B6085127144AB70851BDC706DE
S123C180BDC5E6B108512705B6085120F07D08662765FE081109FF08112609FE080FFF08E4
S123C1A0117A0813FE085F09FF085F264AFE0863FF085FFE080FFF08118605B70813BDC3B8
S123C1C0B1B60805270E8101270A810227108103270C2023B6085281A5271C4C2006B608A2
S123C1E05227144AB70852BDC777BDC676B108522705B6085220F0200BBDC3F47D081926A5
S123C200037F081ABDC3FEBDC415BDC42CBDC445BDC3A1BDC3B17D081526037EC105FE0890
S123C2200627F88601B70816BDC5E6B70851BDC676B70852FC0802CE00001A8300592F06F8
S123C24083005A0820F4F708048FF70805FC08021A83005A270D1A83010E27078601B708FA
S123C26065200B7F08657F080EBDC3A12075FC0808FD08717F0870FC0806FD08747F0873FD
S123C280BDC846FC0879FD087CB6087BB7087ECC0000FD0882CC0296FD0884CC1FBEFD086D
S123C2A086BDC893B60804BDC9F4B7087E7F087D7F087C7F08827F08837F0884FC087FFDBE
S123C2C00885B60881B70887BDC893FC0880FD0861FD085DCE000502FF080AFF080C860560
S123C2E0B7080EFC0802270D1A8300B427078601B70866200B7F08667F0813BDC3B1207590
S123C300FC0808FD08717F0870FC0806FD08747F0873BDC846FC0879FD087CB6087BB70862
S123C3207ECC0000FD0882CC0302FD0884CC78B9FD0886BDC893B60804BDCA16B7087E7F13
S123C340087D7F087C7F08827F08837F0884FC087FFD0885B60881B70887BDC893FC088005
S123C360FD0863FD085FCE000502FF080FFF08118605B708137D081526FB7EC105860FC633
S123C38000BDC498860CC601BDC498860BC607BDC498860AC608BDC4988609C677BDC4983B
S123C3A039F6080E4FC3CB638FE6008608BDC49839F608134FC3CB638FE600FA0814860439
S123C3C0BDC49839B6081484FC8A012019B6081484FC8A022010B6081484FC8A032007B627
S123C3E0081484FC2000B70814398DD88DC3398DDC8DBE398DE08DB9398DE48DB439FC08BB
S123C40002CE000A02F7081C8FCE000A02F7081D8FF7081E39FC0806CE000A02F7081F8F26
S123C420CE000A02F708208FF70821398605F6081CBDC4988606F6081DBDC4988607F6080E
S123C4401EBDC498398601F6081FBDC4988602F60820CA80BDC4988603F60821BDC49839A8
S123C4608601F6081FBDC4988602F60820BDC4988603F60821BDC498394FCE000A02378F53
S123C480CE000A02378F8607BDC498338606BDC498338605BDC4983936373C183CCE10008F
S123C4A01D00021D00041D000118CE00100524051C000120031D00011C00021D000218093A
S123C4C026EB1C0004183838333239FD0802CC0000FD0806BDC3FEBDC415BDC42CBDC4459C
S123C4E0BDC3EF20FE860AB7085B8602BDC8198601BDC8198601BDC819862FBDC8198600B8
S123C500BDC8198633BDC819CE085386FFB7081718FE084818BC084A26107D081726F57AAB
S123C520085B26C6CC000A7EC4CB18A600A70008188C0847260418CE0837180818FF08488F
S123C5408C085726C6B608538102261BB60854810126144FCE0853AB00088C085626F8A189
S123C560002604B60855397A085B27037EC4E5CC00017EC4CBB70822860AB7085B8601BD6A
S123C580C8198604BDC8198601BDC819862FBDC8198600BDC819B60822BDC819B608228B09
S123C5A035BDC81918FE084886FFB7081718BC084A26107D081726F57A085B26C0CC000B36
S123C5C07EC4CB18A600188C0847260418CE0837180818FF08488106270B7A085B269ECC9D
S123C5E000037EC4CB39860AB7085B8602BDC8198601BDC8198600BDC819867CBDC81986AF
S123C6007EBDC81986FDBDC819CE085386FFB7081718FE084818BC084A26107D081726F5DC
S123C6207A085B26C6CC000C7EC4CB18A600A70008188C0847260418CE0837180818FF085A
S123C640488C085726C6B608538102261BB60854810126144FCE0853AB00088C085626F8E1
S123C660A1002604B60855397A085B27037EC5E6CC00047EC4CB860AB7085B8602BDC819C2
S123C6808601BDC8198600BDC819867DBDC819867EBDC81986FEBDC819CE085386FFB7087B
S123C6A01718FE084818BC084A26107D081726F57A085B26C6CC000D7EC4CB18A600A700D2
S123C6C008188C0847260418CE0837180818FF08488C085726C6B608538102261BB60854C7
S123C6E0810126144FCE0853AB00088C085626F8A1002604B60855397A085B27037EC67B6A
S123C700CC00057EC4CBB70822860AB7085B8601BDC8198604BDC8198600BDC819867CBD7C
S123C720C819867EBDC819B60822BDC819B608228BFFBDC81918FE084886FFB7081718BC57
S123C740084A26107D081726F57A085B26C0CC000E7EC4CB18A600188C0847260418CE0823
S123C76037180818FF08488106270B7A085B269ECC00067EC4CB39B70822860AB7085B8674
S123C78001BDC8198604BDC8198600BDC819867DBDC819867EBDC819B60822BDC819B6082B
S123C7A0228B00BDC81918FE084886FFB7081718BC084A26107D081726F57A085B26C0CCC7
S123C7C0000F7EC4CB18A600188C0847260418CE0837180818FF08488106270B7A085B26F6
S123C7E09ECC00077EC4CB3918CE0005CE000A02378F180926F618CE0005328B308D1A181F
S123C8000926F7393684F044444444BDC81132840F8B3081392F028B07183C18FE083618A8
S123C820A700188C0833260418CE0823180818BC083427FA18FF083618383936860D8DD9D5
S123C840860A8DD5323937363CCE08736F036F046F056F066F076F088603B70867A602274C
S123C86028F608723DE307ED0724066C0626026C05A602F608713DE306ED0624026C05A65F
S123C88002F608703DE305ED05097A086726CE3832333937363C183C7F087F7F08807F08C0
S123C8A081C60618CE0882186D00260A5A2704180820F47EC9EEF7086B86FF50C30887186B
S123C8C08F8603CE087C6D0026064A27E60820F6FF0868B7086AB0086B2ED818E601E1003B
S123C8E025034A18091640B7086E81042EC586FFC30881FD086CFE0868B6086A4A2721B785
S123C900086718EC011AA30025132217B608674A271518E603E1022504C60120157EC9B3C3
S123C9207EC9D1B608674AEE004D27010818EC01028FF7086FFE086CEB00E700F6086AF75A
S123C9400867FE0868A600F6086F3DFD088818EC00B3088818ED007A0867273DFE0868A66C
S123C96001F6086F3DFD088818EC01B3088818ED012403186A007A0867271EFE0868A60240
S123C980F6086F3DFD088818EC02B3088818ED022407CDEE0009CDEF0018EC0027084D27BA
S123C9A00FFE0868201718087A086E2D417C086D7EC8F67A086E2D367C086D1808E6004F7B
S123C9C08F0818EC0027DF028F4D2702C6F07EC932E6004F8FCDAC00230C7A086E2D0F7C68
S123C9E0086D180820EF18EC00028F7EC932183838323339F60805270CC1012710C1022742
S123CA0004C1032708B70822865AB00822164FC3CB6F8FA60039F608052714C1012708C1C0
S123CA2002270CC1032700B70822865AB00822164FC3CB6F8FA60039CE10008640A7257D7A
S123CA40081727037A08177C0818B60818813E260B7F0818B608198801B708197C081BB662
S123CA60081B810C27013B7F081BA608B70800843C813C275A840C810C272981082617FC63
S123CA800802C300011A8301682606CC0000FD0802FD0802200EFC08028300012A03CC0106
S123CAA067FD0802B6080084308130272281202611FC08061A8303E72715C30001FD080624
S123CAC0200DFC08062708830001FD08062000A600840826078601B7081520037F081520A4
S123CAE035CE1000A62EB7084C84202608B6084C848026223BA62F18FE084A18A700188C3D
S123CB000847260418CE0837180818FF084AB6084C848026013B18FE083418BC0836273FB0
S123CB201F2E80FC3CCE00085F18A600364424015C0926F93238C40126051D2C4020031CB4
S123CB402C40A72F188C0833260418CE0823180818FF083418BC083627051C2D8020031DBB
S123CB602D803B000424343C7C0004201008400004090D12161B1F23282C3135393E4246E1
S123CB804B4F53575B6064686C7074787C7F83878B8F9296999DA0A4A7ABAEB1B4B7BABEA9
S123CBA0C0C3C6C9CCCED1D3D6D8DBDDDFE1E3E5E7E9EBECEEF0F1F3F4F5F6F7F8F9FAFB0E
S10DCBC0FCFDFDFEFEFEFFFFFFFF7B
S123FF008E01FFCE10008691A7398600A7248600A7358E03FF8605A75D8600A75E8601A7EF
S110FF205F861FA7038600A7027EC0003B7A
S123FFD6CAE1FF2CFF2CFF2CFF2CFF2CFF2CFF2CFF2CFF2CFF2CFF2CFF2CCA38FF2CFF2C00
S10DFFF6FF2CFF2CFF2CFF2CFF0052
S9030000FC
